:0600000083018B018A015F
:06000600850186018C015A
:06000C009D018F0190012F
:060012009101920193012F
:060018009401950198011E
:06001E0099019A01AB01FB
:06002400AC01AA018316E5
:06002A0010308500FF30DC
:0600300086008117640048
:06003600A73081008312D7
:06003C008501860105119B
:06004200051085101530C9
:060048009E009F019F0BCA
:06004E0026289E0B262867
:060054000F30860530307C
:06005A00860483160F303E
:0600600006058600831274
:060066000515051107302D
:06006C009E009F019F0BA6
:0600720038289E0B38281F
:0600780005150511013021
:06007E009E009F019F0B94
:0600840041289E0B4128FB
:06008A000F308605203056
:06009000860405150511B0
:060096002830F8200830BC
:06009C00F8200130F820FD
:0600A2000C30F8200630CE
:0600A800F8200730A10062
:0600AE001321A40008303C
:0600B400A1001321A500CC
:0600BA000B30A100132130
:0600C00003192A150F30A0
:0600C600A1001321031943
:0600CC008D284530E520FF
:0600D2004530E5202D3051
:0600D800E5204930E5209F
:0600DE004E30E520493020
:0600E400E5205430E52088
:0600EA003A30E5200B2175
:0600F0000030A100210810
:0600F6008900B62088001D
:0600FC001C214030803899
:06010200F820C7202108CF
:06010800A520E5200B21FB
:06010E0021080F3C031C58
:060114008D28A10A7A28E3
:06011A000130F820061C74
:060120003F2A712982074D
:06012600003400340A342D
:06012C00003400346434CD
:0601320000340334E83440
:06013800003427341034EE
:06013E0001348634A034F8
:060144000F344234403488
:06014A008207303431345D
:0601500032343334343474
:0601560035343634373465
:06015C003834393441344F
:0601620042344334443432
:0601680045344634820715
:06016E000D34BC343634F0
:060174000D34BB340A3417
:06017A00003414340134CE
:0601800000340034FF34DE
:06018600FF3428340A34A6
:06018C0000348316F03080
:060192000604860018308F
:0601980085008312051032
:06019E008514051506089A
:0601A400F0399B0005117B
:0601AA0000000000051535
:0601B0000511060E0F39D7
:0601B6001B049B1BC7287F
:0601BC00851083160F30D0
:0601C20006058600831211
:0601C80008009600C720AC
:0601CE000F308605160843
:0601D400F03986048510DD
:0601DA00051405150511D6
:0601E0000F308605160E2B
:0601E600F0398604051546
:0601EC0005110800960059
:0601F200C7200F30860556
:0601F8001608F039860430
:0601FE0085100510051537
:0602040005110F30860514
:06020A00160EF039860417
:06021000051505110800B0
:06021600FF309E009F0175
:06021C009F0B0E299E0B52
:060222000E290800831202
:0602280021088900831685
:06022E0008148312080809
:06023400A2000800831681
:06023A008B13081555307E
:060240008900AA308900CC
:0602460088148818242929
:06024C008B1708002A12C6
:060252000F0893020318DF
:0602580033299403940A0F
:06025E00031D3229950387
:060264009403100894024F
:06026A000318382995037A
:06027000110895020318BD
:060276002A1608002A12FE
:06027C000F089307031CAC
:060282004829940F4829F1
:0602880001309507031888
:06028E002A161008940777
:06029400031C4D29950A30
:06029A001108950703188E
:0602A0002A1608002708E1
:0602A6008F002808900003
:0602AC0029089100080082
:0602B2002A1301301302C3
:0602B80003186329013068
:0602BE001402031863297D
:0602C4002A1708000330B8
:0602CA00861C0030A100BB
:0602D00013219500A10AB4
:0602D60013219400A10AAF
:0602DC001321930008004D
:0602E20000308038F82016
:0602E800C7204530E520AF
:0602EE004530E5202D3033
:0602F400E5203130E52099
:0602FA002E30E520333038
:06030000E5200B210B219A
:060306000B2106080F396F
:06030C00031D7129013000
:06031200F820C720A10144
:06031800A201A301061C76
:06031E009729A10A210845
:060324000F3C031CA101C7
:06032A000B212310861CCC
:060330009B29A20A0B212B
:06033600061D9F29A20331
:06033C000B21861DC02903
:060342000B2121088900D7
:06034800220888001C21C0
:06034E000130F820C72079
:060354002A30E5205330C1
:06035A00E5204130E52022
:060360005630E520453097
:06036600E5204430E52013
:06036C002A30E5200B2100
:060372000B210B210B2101
:060378000130F820C7204F
:06037E00A3014130E5205F
:060384004430E520443086
:06038A00E5205230E520E1
:060390003A30E5202318BD
:06039600CE2913212314FF
:06039C002108F0398E007B
:0603A2000E0EA520E5206F
:0603A80021080F39A52019
:0603AE00E520403080381C
:0603B400F820C7204430D0
:0603BA00E5204130E520C2
:0603C0005430E52041303D
:0603C600E5203A30E520BD
:0603CC002208F0398E004A
:0603D2000E0EA520E5203F
:0603D80022080F39A520E8
:0603DE00E520003080382C
:0603E400F820C7208E295D
:0603EA009B010C089C00C1
:0603F000922098020318A0
:0603F600052A0130990206
:0603FC000318052A013080
:060402009A020318052A0E
:060408001B149C031C08FC
:06040E0092209902031880
:06041400102A01309A02DB
:06041A000318102A1B1458
:060420009C031C08922061
:060426009A020318182AD7
:06042C000314192A1B0C49
:0604320000349B010C08E0
:060438009C0092209807D1
:06043E00031C2A2A013014
:060444009907031C2A2A9F
:06044A0001309A07031CBB
:060450002A2A1B149C0384
:060456001C08922099072A
:06045C00031C352A0130EB
:060462009A07031C352A75
:060468001B149C031C089C
:06046E0092209A07031C16
:060474003D2A03143E2A9C
:06047A001B0C00341130E0
:060480008C0009308D0024
:060486008E0106309D000E
:06048C00F5210318502ABF
:060492008E0A8D03031D1C
:06049800462A03308C022D
:06049E00532A1A2203306C
:0604A4008C0209308D00FE
:0604AA0010301D079B004D
:0604B0009B031B08840001
:0604B6000E088E0180001B
:0604BC009D0301300C0756
:0604C200031D462A180884
:0604C8008F00AA1E692A44
:0604CE0006108611063045
:0604D4009D002108060551
:0604DA00A200A2197C2A19
:0604E00007308038F8200F
:0604E600C7202030E520D4
:0604EC000B308038F820FF
:0604F200C7202030E520C8
:0604F80000308038F820FE
:0604FE00C7208608A100E2
:060504000F301D0784000A
:06050A00000803198B2A12
:060510003038E520942ABA
:0605160006301D02031D6A
:06051C00922A2030E520C8
:06052200942A3030E520B0
:060528002A1D9D2A0C3083
:06052E00A1001321031DD2
:060534009F2AAA17A32A6A
:06053A008619A32AAA1392
:060540000230A600AA2A09
:060546000130A6000A309E
:06054C00A1001321031DB4
:06055200B02A26081D027C
:06055800031DB02A2E3045
:06055E00E5202A1DB52A6C
:06056400AA1BB92AB72A08
:06056A008619B92A0530D4
:06057000BA2A04301D024E
:06057600031DBF2A2E3018
:06057C00E5200930A1009A
:060582001321031DCC2A29
:0605880001301D02031DFD
:06058E00CC2A4030803849
:06059400F820C7209D0BBA
:06059A00822A0A30A100D4
:0605A0001321031DD92AFE
:0605A6000F301D07840068
:0605AC0000083038E520D4
:0605B2002030E5204D3071
:0605B800E5204830E520BB
:0605BE007A30E5202A1D41
:0605C400EC2A2030E520C6
:0605CA002A1CEA2A4C3055
:0605D000E520EC2A2030BA
:0605D600E5200030803832
:0605DC00F82097018101E7
:0605E200000000009D0175
:0605E800C7309E000B303D
:0605EE009F000530A00093
:0605F4008B0110308500B0
:0605FA0083161F3085008E
:0606000083120B1D062B06
:06060600970A0B11092BFD
:06060C00000000000000E8
:060612009E0B012BC73016
:060618009E009F0B012B68
:06061E000B309F00A00B51
:06062400012B06108611F7
:06062A0082308E000B1D62
:060630001C2B970A0B11C0
:060636001F2B0000000074
:06063C0000008E0B172BDD
:0606420024088E008E0B5F
:06064800232B25088E00A3
:06064E0000008E0B272BBB
:06065400030186001030D6
:06065A0085008316173035
:06066000850083120B1956
:06066600970A0B110108C8
:06066C00990017089A0036
:060672009B019B0A8515A7
:0606780085110B110108C1
:06067E00190203193A2BDA
:060684009B0A9B099B0A82
:06068A001B0A980010306D
:0606900085008316043012
:06069600850083122A1DFD
:06069C00CC2B18089300AE
:0606A200190894001A087B
:0606A80095008316F630F8
:0606AE0006058600831220
:0606B4002A18932B0D3003
:0606BA00A10013212B0238
:0606C000031D652BAA18C2
:0606C6006E2B672BAB0A4E
:0606CC00CC2B1808A7006A
:0606D2001908A8001A0837
:0606D800A900AA14522142
:0606DE00282159212A1F0A
:0606E4007D2B0E30A10089
:0606EA0013212C02031D88
:0606F000CB2B2A14AA1016
:0606F600AC01CC2B053025
:0606FC008F009001910146
:060702002A1E8D2BFA30C7
:060708008F00FF3090009D
:06070E00FF3091003D21C7
:060714002A1A902B732B42
:06071A003D212A1A732B99
:06072000AB01AA10CC2B76
:06072600AA125221282155
:06072C0059212A1BC92B14
:0607320013089B002A1AC7
:06073800B82B0614861127
:06073E009B0A0319A42B25
:060744009B0A0319AA162E
:06074A00910190010A304C
:060750008F003D212A1A72
:06075600C92B0E30A100CA
:06075C0013212C02031919
:06076200B42BAC0ACC2B05
:060768002A10AC01AB01F8
:06076E00CC2B06108615DD
:060774009B030319BF2BDB
:06077A009B030319AA16FF
:06078000F6308F00FF308F
:060786009000FF3091001D
:06078C003D212A1AAC2BEE
:06079200AC01CC2BAC0A07
:0607980064210630A100FF
:06079E0013210319FB2BDF
:0607A4000619FB2B1A08E8
:0607AA0091001908900007
:0607B00018088F00051976
:0607B600F42B28212A1A91
:0607BC00F52B6421150875
:0607C2009B0011089500E8
:0607C8001B08910014085B
:0607CE009B0010089400DE
:0607D4001B089000130851
:0607DA009B000F089300D4
:0607E0001B088F00282118
:0607E600F52B3D21150872
:0607EC009A0014089900B8
:0607F200130898003F2AE5
:0607F800FF3FFF3FFF3F41
:0207FE00FF3FBB
:084000000F000F000F000F007C
:02400E00F93F78
:00000001FF
